BL51 BANKED LINKER/LOCATER V6.22                                                        05/25/2017  14:58:10  PAGE 1


BL51 BANKED LINKER/LOCATER V6.22, INVOKED BY:
E:\KEIL-C51\C51\BIN\BL51.EXE ..\OBJ\main.obj, ..\OBJ\LCD drive.obj TO ..\OBJ\9341-16bit PRINT (.\9341-16bit.m51) RAMSIZE
>>  (256)


MEMORY MODEL: COMPACT


INPUT MODULES INCLUDED:
  ..\OBJ\main.obj (MAIN)
  ..\OBJ\LCD drive.obj (LCD_DRIVE)
  E:\KEIL-C51\C51\LIB\C51C.LIB (?C_STARTUP)


LINK MAP OF MODULE:  ..\OBJ\9341-16bit (MAIN)


            TYPE    BASE      LENGTH    RELOCATION   SEGMENT NAME
            -----------------------------------------------------

            * * * * * * *   D A T A   M E M O R Y   * * * * * * *
            REG     0000H     0008H     ABSOLUTE     "REG BANK 0"
            IDATA   0008H     0001H     UNIT         ?STACK

            * * * * * * *  X D A T A   M E M O R Y  * * * * * * *
            XDATA   0000H     001CH     INPAGE       _PDATA_GROUP_

            * * * * * * *   C O D E   M E M O R Y   * * * * * * *
            CODE    0000H     0003H     ABSOLUTE     
            CODE    0003H     0601H     UNIT         ?CO?LCD_DRIVE
            CODE    0604H     023EH     UNIT         ?PR?LCD_INIT?LCD_DRIVE
            CODE    0842H     00ECH     UNIT         ?PR?_GUI_SPRINTF_CHAR?LCD_DRIVE
            CODE    092EH     0064H     UNIT         ?PR?_GUI_SPRINTF_STRING?LCD_DRIVE
            CODE    0992H     004BH     UNIT         ?PR?_LCD_TEST_SINGLECOLOR?LCD_DRIVE
            CODE    09DDH     0047H     UNIT         ?PR?_LCD_SETWINDOW?LCD_DRIVE
            CODE    0A24H     003CH     UNIT         ?PR?MAIN?MAIN
            CODE    0A60H     0036H     UNIT         ?PR?DISPLAY_ID?LCD_DRIVE
            CODE    0A96H     0025H     UNIT         ?PR?_DELAYMS?LCD_DRIVE
            CODE    0ABBH     001EH     UNIT         ?PR?_LLCD_WRITE_DATA?LCD_DRIVE
            CODE    0AD9H     001BH     UNIT         ?PR?HD_RESET?LCD_DRIVE
            CODE    0AF4H     001BH     UNIT         ?PR?_LLCD_WRITE_CMD?LCD_DRIVE
            CODE    0B0FH     0014H     UNIT         ?PR?_GUI_POINT?LCD_DRIVE
            CODE    0B23H     0014H     UNIT         ?PR?_LCD_SETXY?LCD_DRIVE
            CODE    0B37H     000CH     UNIT         ?PR?_DELAYUS?LCD_DRIVE
            CODE    0B43H     000CH     UNIT         ?C_C51STARTUP



OVERLAY MAP OF MODULE:   ..\OBJ\9341-16bit (MAIN)


SEGMENT                                       PDATA_GROUP
  +--> CALLED SEGMENT                       START    LENGTH
-----------------------------------------------------------
?C_C51STARTUP                               -----    -----
  +--> ?PR?MAIN?MAIN

?PR?MAIN?MAIN                               -----    -----
BL51 BANKED LINKER/LOCATER V6.22                                                      05/25/2017  14:58:10  PAGE 2


  +--> ?PR?HD_RESET?LCD_DRIVE
  +--> ?PR?LCD_INIT?LCD_DRIVE
  +--> ?PR?_DELAYMS?LCD_DRIVE
  +--> ?PR?_LCD_TEST_SINGLECOLOR?LCD_DRIVE
  +--> ?PR?DISPLAY_ID?LCD_DRIVE

?PR?HD_RESET?LCD_DRIVE                      -----    -----
  +--> ?PR?_DELAYMS?LCD_DRIVE

?PR?_DELAYMS?LCD_DRIVE                      0000H    0002H
  +--> ?PR?_DELAYUS?LCD_DRIVE

?PR?LCD_INIT?LCD_DRIVE                      -----    -----
  +--> ?PR?_LLCD_WRITE_CMD?LCD_DRIVE
  +--> ?PR?_LLCD_WRITE_DATA?LCD_DRIVE
  +--> ?PR?_DELAYMS?LCD_DRIVE
  +--> ?PR?_LCD_TEST_SINGLECOLOR?LCD_DRIVE

?PR?_LCD_TEST_SINGLECOLOR?LCD_DRIVE         0000H    0002H
  +--> ?PR?_LCD_SETWINDOW?LCD_DRIVE

?PR?_LCD_SETWINDOW?LCD_DRIVE                0016H    0006H
  +--> ?PR?_LLCD_WRITE_CMD?LCD_DRIVE
  +--> ?PR?_LLCD_WRITE_DATA?LCD_DRIVE

?PR?DISPLAY_ID?LCD_DRIVE                    -----    -----
  +--> ?CO?LCD_DRIVE
  +--> ?PR?_GUI_SPRINTF_STRING?LCD_DRIVE

?PR?_GUI_SPRINTF_STRING?LCD_DRIVE           0000H    0009H
  +--> ?PR?_GUI_SPRINTF_CHAR?LCD_DRIVE

?PR?_GUI_SPRINTF_CHAR?LCD_DRIVE             0009H    000BH
  +--> ?CO?LCD_DRIVE
  +--> ?PR?_GUI_POINT?LCD_DRIVE

?PR?_GUI_POINT?LCD_DRIVE                    0014H    0002H
  +--> ?PR?_LCD_SETXY?LCD_DRIVE
  +--> ?PR?_LLCD_WRITE_DATA?LCD_DRIVE

?PR?_LCD_SETXY?LCD_DRIVE                    -----    -----
  +--> ?PR?_LCD_SETWINDOW?LCD_DRIVE



SYMBOL TABLE OF MODULE:  ..\OBJ\9341-16bit (MAIN)

  VALUE           TYPE          NAME
  ----------------------------------

  -------         MODULE        MAIN
  C:0000H         SYMBOL        _ICE_DUMMY_
  D:0090H         PUBLIC        P1
  D:00B0H         PUBLIC        P3
  D:00A8H         PUBLIC        IE
  D:00B8H         PUBLIC        IP
  C:0A24H         PUBLIC        main
BL51 BANKED LINKER/LOCATER V6.22                                                      05/25/2017  14:58:10  PAGE 3


  D:0098H         PUBLIC        SCON
  D:0088H         PUBLIC        TCON
  D:00C8H         PUBLIC        T2CON
  D:00D0H         PUBLIC        PSW
  -------         PROC          MAIN
  C:0A24H         LINE#         14
  C:0A24H         LINE#         15
  C:0A24H         LINE#         17
  C:0A27H         LINE#         18
  C:0A2AH         LINE#         19
  C:0A2AH         LINE#         20
  C:0A2AH         LINE#         22
  C:0A38H         LINE#         23
  C:0A3FH         LINE#         24
  C:0A4DH         LINE#         25
  C:0A54H         LINE#         26
  C:0A5BH         LINE#         27
  C:0A5EH         LINE#         28
  -------         ENDPROC       MAIN
  -------         ENDMOD        MAIN

  -------         MODULE        LCD_DRIVE
  C:0000H         SYMBOL        _ICE_DUMMY_
  D:0080H         PUBLIC        P0
  D:0090H         PUBLIC        P1
  D:00A0H         PUBLIC        P2
  D:00B0H         PUBLIC        P3
  C:0ABEH         PUBLIC        _LLCD_WRITE_DATA
  D:00A8H         PUBLIC        IE
  C:0AD9H         PUBLIC        HD_reset
  D:00B8H         PUBLIC        IP
  C:09DDH         PUBLIC        _LCD_setwindow
  B:0090H.1       PUBLIC        RS
  D:0098H         PUBLIC        SCON
  D:0088H         PUBLIC        TCON
  C:0992H         PUBLIC        _LCD_TEST_SingleColor
  C:0AF4H         PUBLIC        _LLCD_WRITE_CMD
  C:0A60H         PUBLIC        Display_ID
  C:092EH         PUBLIC        _GUI_sprintf_string
  C:0014H         PUBLIC        font16x8
  C:0842H         PUBLIC        _GUI_sprintf_char
  C:0B0FH         PUBLIC        _GUI_Point
  B:0090H.3       PUBLIC        RDB
  B:0090H.0       PUBLIC        TFT_CS
  D:00C8H         PUBLIC        T2CON
  C:0604H         PUBLIC        LCD_init
  B:0090H.4       PUBLIC        RES
  B:0090H.2       PUBLIC        WRB
  C:0A96H         PUBLIC        _delayms
  C:0B23H         PUBLIC        _LCD_setxy
  D:00D0H         PUBLIC        PSW
  C:0B37H         PUBLIC        _delayus
  -------         PROC          DISPLAY_ID
  C:0A60H         LINE#         10
  C:0A60H         LINE#         11
  C:0A60H         LINE#         13
  C:0A7BH         LINE#         14
BL51 BANKED LINKER/LOCATER V6.22                                                      05/25/2017  14:58:10  PAGE 4


  -------         ENDPROC       DISPLAY_ID
  -------         PROC          LCD_INIT
  C:0604H         LINE#         21
  C:0604H         LINE#         22
  C:0604H         LINE#         24
  C:060BH         LINE#         25
  C:060EH         LINE#         26
  C:0615H         LINE#         27
  C:061CH         LINE#         29
  C:0623H         LINE#         30
  C:062AH         LINE#         31
  C:0631H         LINE#         32
  C:0638H         LINE#         33
  C:063FH         LINE#         35
  C:0646H         LINE#         36
  C:064DH         LINE#         37
  C:0654H         LINE#         38
  C:065BH         LINE#         40
  C:0662H         LINE#         41
  C:0669H         LINE#         42
  C:0670H         LINE#         43
  C:0673H         LINE#         44
  C:067AH         LINE#         45
  C:0681H         LINE#         47
  C:0688H         LINE#         48
  C:068FH         LINE#         50
  C:0696H         LINE#         51
  C:069CH         LINE#         52
  C:06A2H         LINE#         54
  C:06A9H         LINE#         55
  C:06B0H         LINE#         57
  C:06B7H         LINE#         58
  C:06BEH         LINE#         60
  C:06C5H         LINE#         61
  C:06CCH         LINE#         62
  C:06D3H         LINE#         64
  C:06DAH         LINE#         65
  C:06E1H         LINE#         67
  C:06E8H         LINE#         68
  C:06EFH         LINE#         70
  C:06F6H         LINE#         71
  C:06FDH         LINE#         73
  C:0704H         LINE#         74
  C:070AH         LINE#         75
  C:0711H         LINE#         77
  C:0718H         LINE#         78
  C:071FH         LINE#         79
  C:0726H         LINE#         81
  C:072DH         LINE#         82
  C:0733H         LINE#         84
  C:073AH         LINE#         85
  C:0741H         LINE#         87
  C:0748H         LINE#         88
  C:074FH         LINE#         89
  C:0756H         LINE#         90
  C:075DH         LINE#         91
  C:0764H         LINE#         92
BL51 BANKED LINKER/LOCATER V6.22                                                      05/25/2017  14:58:10  PAGE 5


  C:076BH         LINE#         93
  C:0772H         LINE#         94
  C:0779H         LINE#         95
  C:0780H         LINE#         96
  C:0787H         LINE#         97
  C:078EH         LINE#         98
  C:0795H         LINE#         99
  C:079CH         LINE#         100
  C:07A3H         LINE#         101
  C:07AAH         LINE#         102
  C:07B0H         LINE#         103
  C:07B7H         LINE#         104
  C:07BDH         LINE#         105
  C:07C4H         LINE#         106
  C:07CBH         LINE#         107
  C:07D2H         LINE#         108
  C:07D9H         LINE#         109
  C:07E0H         LINE#         110
  C:07E7H         LINE#         111
  C:07EEH         LINE#         112
  C:07F5H         LINE#         113
  C:07FCH         LINE#         114
  C:0803H         LINE#         115
  C:080AH         LINE#         116
  C:0811H         LINE#         117
  C:0818H         LINE#         118
  C:081FH         LINE#         120
  C:0826H         LINE#         121
  C:082DH         LINE#         122
  C:0834H         LINE#         123
  C:083BH         LINE#         124
  -------         ENDPROC       LCD_INIT
  -------         PROC          HD_RESET
  C:0AD9H         LINE#         132
  C:0AD9H         LINE#         133
  C:0AD9H         LINE#         134
  C:0ADBH         LINE#         135
  C:0AE2H         LINE#         136
  C:0AE4H         LINE#         137
  C:0AEBH         LINE#         138
  C:0AEDH         LINE#         139
  -------         ENDPROC       HD_RESET
  -------         PROC          _LLCD_WRITE_CMD
  D:0004H         SYMBOL        cmd
  C:0AF4H         LINE#         146
  C:0AF8H         LINE#         147
  C:0AF8H         LINE#         149
  C:0AFAH         LINE#         150
  C:0AFCH         LINE#         151
  C:0AFEH         LINE#         152
  C:0B00H         LINE#         153
  C:0B04H         LINE#         154
  C:0B08H         LINE#         155
  C:0B0AH         LINE#         156
  C:0B0CH         LINE#         157
  C:0B0EH         LINE#         159
  -------         ENDPROC       _LLCD_WRITE_CMD
BL51 BANKED LINKER/LOCATER V6.22                                                      05/25/2017  14:58:10  PAGE 6


  -------         PROC          L?0045
  -------         ENDPROC       L?0045
  -------         PROC          _LLCD_WRITE_DATA
  D:0004H         SYMBOL        dataa
  C:0ABEH         LINE#         164
  C:0AC2H         LINE#         165
  C:0AC2H         LINE#         167
  C:0AC4H         LINE#         168
  C:0AC6H         LINE#         169
  C:0AC8H         LINE#         170
  C:0ACAH         LINE#         171
  C:0ACEH         LINE#         172
  C:0AD2H         LINE#         173
  C:0AD4H         LINE#         174
  C:0AD6H         LINE#         175
  C:0AD8H         LINE#         177
  -------         ENDPROC       _LLCD_WRITE_DATA
  -------         PROC          _GUI_SPRINTF_STRING
  X:0000H         SYMBOL        x
  X:0001H         SYMBOL        y
  X:0003H         SYMBOL        s
  X:0005H         SYMBOL        color
  X:0007H         SYMBOL        b_color
  C:092EH         LINE#         183
  C:093EH         LINE#         184
  C:093EH         LINE#         185
  C:094DH         LINE#         186
  C:094DH         LINE#         187
  C:097EH         LINE#         188
  C:0984H         LINE#         189
  C:0991H         LINE#         192
  -------         ENDPROC       _GUI_SPRINTF_STRING
  -------         PROC          _GUI_SPRINTF_CHAR
  X:0009H         SYMBOL        x
  X:000AH         SYMBOL        y
  X:000CH         SYMBOL        c
  X:000DH         SYMBOL        color
  X:000FH         SYMBOL        b_color
  -------         DO            
  X:0011H         SYMBOL        s_x
  X:0012H         SYMBOL        s_y
  X:0013H         SYMBOL        temp
  D:0006H         SYMBOL        j
  -------         ENDDO         
  C:0842H         LINE#         197
  C:084FH         LINE#         198
  C:084FH         LINE#         201
  C:0853H         LINE#         202
  C:0863H         LINE#         203
  C:0863H         LINE#         204
  C:087CH         LINE#         205
  C:087CH         LINE#         206
  C:0881H         LINE#         207
  C:0894H         LINE#         208
  C:08A3H         LINE#         210
  C:08B0H         LINE#         211
  C:08B0H         LINE#         212
BL51 BANKED LINKER/LOCATER V6.22                                                      05/25/2017  14:58:10  PAGE 7


  C:08C4H         LINE#         213
  C:08C4H         LINE#         214
  C:08E9H         LINE#         215
  C:08E9H         LINE#         216
  C:08FBH         LINE#         217
  C:08FDH         LINE#         219
  C:08FDH         LINE#         220
  C:091EH         LINE#         221
  C:091EH         LINE#         222
  C:091EH         LINE#         223
  C:0925H         LINE#         224
  C:0925H         LINE#         225
  C:092DH         LINE#         226
  -------         ENDPROC       _GUI_SPRINTF_CHAR
  -------         PROC          _GUI_POINT
  D:0007H         SYMBOL        x
  D:0004H         SYMBOL        y
  X:0014H         SYMBOL        color
  C:0B0FH         LINE#         231
  C:0B16H         LINE#         232
  C:0B16H         LINE#         233
  C:0B19H         LINE#         234
  -------         ENDPROC       _GUI_POINT
  -------         PROC          _LCD_SETXY
  D:0006H         SYMBOL        x
  D:0082H         SYMBOL        y
  C:0B23H         LINE#         240
  C:0B29H         LINE#         241
  C:0B29H         LINE#         242
  -------         ENDPROC       _LCD_SETXY
  -------         PROC          _LCD_SETWINDOW
  D:0002H         SYMBOL        x0
  X:0017H         SYMBOL        y0
  D:0003H         SYMBOL        x1
  X:001AH         SYMBOL        y1
  C:09DDH         LINE#         248
  C:09E6H         LINE#         249
  C:09E6H         LINE#         250
  C:09EDH         LINE#         251
  C:09F2H         LINE#         252
  C:09F7H         LINE#         253
  C:09FCH         LINE#         254
  C:0A01H         LINE#         256
  C:0A06H         LINE#         257
  C:0A0CH         LINE#         258
  C:0A12H         LINE#         259
  C:0A19H         LINE#         260
  C:0A1FH         LINE#         262
  -------         ENDPROC       _LCD_SETWINDOW
  -------         PROC          _LCD_TEST_SINGLECOLOR
  X:0000H         SYMBOL        color
  -------         DO            
  D:0004H         SYMBOL        i
  D:0002H         SYMBOL        j
  -------         ENDDO         
  C:0992H         LINE#         268
  C:0999H         LINE#         269
BL51 BANKED LINKER/LOCATER V6.22                                                      05/25/2017  14:58:10  PAGE 8


  C:0999H         LINE#         272
  C:09ABH         LINE#         274
  C:09ADH         LINE#         275
  C:09AFH         LINE#         276
  C:09B1H         LINE#         278
  C:09B4H         LINE#         279
  C:09B4H         LINE#         280
  C:09B7H         LINE#         281
  C:09B7H         LINE#         282
  C:09BCH         LINE#         283
  C:09C0H         LINE#         284
  C:09C2H         LINE#         285
  C:09C4H         LINE#         286
  C:09CFH         LINE#         287
  C:09DAH         LINE#         289
  C:09DCH         LINE#         290
  -------         ENDPROC       _LCD_TEST_SINGLECOLOR
  -------         PROC          _DELAYMS
  X:0000H         SYMBOL        value
  C:0A96H         LINE#         296
  C:0A9DH         LINE#         297
  C:0A9DH         LINE#         298
  C:0AA6H         LINE#         299
  C:0AA6H         LINE#         300
  C:0AADH         LINE#         301
  C:0AB8H         LINE#         302
  C:0ABAH         LINE#         303
  -------         ENDPROC       _DELAYMS
  -------         PROC          _DELAYUS
  D:0006H         SYMBOL        value1
  C:0B37H         LINE#         308
  C:0B37H         LINE#         309
  C:0B37H         LINE#         310
  C:0B3BH         LINE#         311
  C:0B42H         LINE#         312
  -------         ENDPROC       _DELAYUS
  -------         ENDMOD        LCD_DRIVE

Program Size: data=9.0 xdata=28 code=2895
LINK/LOCATE RUN COMPLETE.  0 WARNING(S),  0 ERROR(S)
